S12301007E012C486561646572203D200420416C6C6F63203D20042020526F6F74203D2079
S10B0120044572726F722004A1
S123012CBDC02186F09702BD202E27037E02717F01287F01297F012A7F012BCE0103BDC0E7
S123014C09CE012ABDC015BDC021BD027DCE1000864DB710008643B710018646B7100286FD
S123016C53B710038602B71004CE0000FF1005CEFFFFFF1007CE5555FF1009CE0001FF10CD
S123018C2BCE0080FF102DCE0081FF102FCE0088FF1031CE1000BD201727037E0271CE01BB
S12301AC0DBDC0097C012BCE012ABDC015BD027D5FCE1000C18A22066C00085C20F6CE10B9
S12301CC00BD2017BD027D7C012B5FC17D2211CE1000BD201727037E02717C012B5C20EB6B
S12301EC862DBDC0038620BDC003CE012ABDC015BDC021CE0117BDC0097C012BCE012ABDA3
S123020CC015BD027DCE1000BD20177C012BCE1000BD20177C012BCE1000BD20177C012B4F
S123022CCE1000BD20177C012BCE1000BD20177C012BCE1000BD20177C012BCE1000BD2085
S123024C177C012BCE1000BD201727037E0271862DBDC0038620BDC003CE012ABDC015BD41
S122026CC0217EC000CE0121BDC009BDC0217EC000CE10008C120022056F000820F63995
S1232000BD2053BD205BBD20708601B79FD28620B79FD77E208D39BD2053BD205BBD20706C
S12320208601B79FD28630B79FD77E20A539BD2035BD2063398604B79FD7BD2053BD205BE4
S123204086E0B79FD68601B79FD186EFB79FD7BD205339B69FD7858026F939B69FD78540B7
S123206027F939B69FD785012704B69FD1394F39B6012BB79FD3B6012AB79FD4B60129B792
S12320809FD5B60128840F8AE0B79FD639BD2053B69FD78508270CB69FD0A70008BD206357
S12020A027EB394F39BD2053B69FD78508270CA600B79FD008BD206327EB394F3949
S9030000FC
